:02000000805E20
:1000600053D74175817F759E82759D09759852752C
:10007000310451F375A080780075400775410EC2B8
:1000800090C291C2927520002092FD2091FDE2B4B1
:10009000080320910971452091FDE2B408237406FC
:1000A0002090FDF22091FDE2B44C0553D74280062A
:1000B000B4480353D74175331851E931D851F3800f
:1000C000D6B407115156B40E0C5156F537F53251CE
:1000D00056F5388004714580BEB4452479407B06CE
:1000E0002091FDE2F709DBF8E5447002747CF53AF3
:1000F00051E9313951F37145E5352090FDF2809792
:10010000B4571051E9313951F37145E5352090FD6F
:10011000F28084B4561051E9313951F37145E53517
:100120002090FDF20197B452AC51E9313951F3718D
:1001300045E5352090FDF20197C0D0C200C204C24F
:1001400003517BE531518D30000B711E9003E65158
:100150006C711E806D7539007407518D20006374B9
:100160000E518D20005CE537518DD204200053E5FF
:1001700038518D20004CB4451579407B06E7518DF0
:1001800020003F09DBF7AF3A717ADFFC8022AA3208
:100190007DFA209103E2800FDDF8711E9004785102
:0901A0006C711ED203801B518D0D
:1001A9007DFA200014DAE25184716F517BE5310444
:1001B900518D20000451B1F5355184300305753551
:1001C90007C204300006753507D0D022D0D022C02E
:1001D90002C0D0C200753664517BE531518D3000C3
:1001E9001851847150D536F074082090FDF2F53518
:1001F900900433516C711E803D7408518D30000993
:10020900900449516C711E802D5184716F517BE5A9
:100219003104518D30000B900459516C711E8016B8
:100229007A1751CD2090FDF27185DAF651B12090FF
:10023900FDF27185711E518430000D74072090FD07
:10024900F2F535D0D0D00222D0D0D002222091FDB3
:10025900E2222090FDF222E49360072090FDF2A3B0
:1002690080F522E493600A3099FDC299F599A3803B
:10027900F222D2EEC200C2EFC2ED22D2EEC2EFD21A
:10028900EDD2EF22C0E0C200753008D2EEC2ED33E4
:1002990092EFD2ED00C2EDD530F5C2EED2ED30ECE1
:1002A90002D200C2EDD0E022753008C2EEC2EDD212
:1002B900EDC2EDA2EC33D530F6D2EED2EFD2EDC2DB
:0B02C900EDC2EE22753008C2EEC2ED5F
:1002D400D2EDC2EDA2EC33D530F6D2EEC2EFD2EDC0
:1002E400C2EDC2EE2275E8A8C200C201D2ED2275A9
:1002F400E80022C0F0C0D075F0648424302090FD62
:10030400F2E5F075F00A8424302090FDF2E5F02443
:10031400302090FDF2D0D0D0F022740D7185740A93
:10032400718522C0E0C0D0F5F0C4540F718D718581
:10033400E5F0540F718D718574207185D0D0D0E0B3
:1003440022C0E0209103E280FAD0E022C0037B3295
:100354007164DBFCD00322C0037B20DBFED00322CC
:10036400C0037B29715BDBFCD00322C0037B647177
:100374005BDBFCD00322C0037B057164DBFCD00390
:10038400223099FDC299F59922540FB40A00400213
:100394002407243022C0D0C39004CD516CE53971B8
:1003A40027711EE960329003FF516CE7091539711A
:1003B40027711EE96022900416516CE70915397102
:1003C40085711E30040F900420516CAC39E77127FD
:1003D40009DCFA711ED0D0229004B0516C711ED089
:1003E400D0224E6F2041434B20666F7220736C61A4
:1003F40076652061646472657373004672616D652D
:100404002D4C656E6774682066726F6D2050433A98
:100414002000436F6D6D616E643A20004672616D19
:10042400653A20004572726F722061743A20004E62
:100434006F20636F6E6E65637420746F204932435E
:100444002041524D004E6F2041434B20666F722075
:1004540030783038004E6F2041434B20666F722055
:1004640052656164205265717565737420537472AA
:10047400696E670054696D654F7574205553422049
:100484004932432D4672616D65004C656176652085
:10049400496E690054696D654F7574205553422047
:1004A400496E707574204672616D65004E6F206DE3
:1004B4006F7265206461746120696E206465627581
:1004C400672062756666657200427974657320748C
:1004D4006F204932432073656E646564203A0030AE
:1004E4007830382073656E64656E2C203234204277
:1004F40079746520656D7066616E67656E0052750E
:100504006E2073656E64656E2C20312042797465AB
:1005140020656D7066616E67656E00322042797485
:1005240065732073656E64656E2C20322042797485
:10053400657320656D7066616E67656E00646174D5
:1005440061207472616E73666572206572726F7277
:100554003A20004144754337303236202044363245
:0C0564002020443359202020200A0D00E4
:00000001FF
